:0E000000802EFF022D9EFFFFFFFFFF021E1B42
:0300230002024D89
:20002E0034147581227508FF7509BF90AC98E4F0124EF180ED12001B80FBC82581C822C96A
:20004E002581C97A0022D083D082CF2581F581CFC082C08322CF2581F581CF22FBE0CB22DD
:20006E00FCE0FBA3E0CC22FAE0F9A3E0CA2229F9E5F03AFA227C00CB30E7011CCB2275F0CE
:20008E000030E70215F022FDE493A3FEE493A3FF4E7009E493FE740193FF800BE493A3B547
:2000AE00050BE493B5F0068F838E82E473A380D8FEEBA4FD8EF0ECA4FCEB8EF0A4C5F02C0A
:2000CE002DC5F02211D88EF0ED22C002C001AAF0F97E007D007F11C3E933F9EA33FADF0821
:2000EE00F5F0E9D001D00222ED33FDEE33FEC3ED9BF5F0EE9C40E0ADF0FED380DBBB0001C4
:20010E0022C333C5F033C5F0DBF722BB000122C3C5F013C5F013DBF722240280022401C571
:20012E00F03400C5F022C394028003C39401C5F09400C5F0223139F4C5F0F4C5F02245F04F
:20014E0070220422319B4024801A319B401E7014801A319B400E7014800A319B500E8004F1
:20016E0031AF6008E4F5F02231AF60F8E4F5F0042231AF40F780ED31AF40F170E780ED318D
:20018E00AF40E170E780DD31AF50E180D7C39BC5F09C20E70720D207C345F02220D2F9D3D7
:2001AE0022C5F0C39C7003E5F09B2290AC98E0A360EEE0FFA3E0A3CF2582F582EF3583F5C3
:2001CE008380EB7E00CF2508F582EE3509F583EF227E00CF2508F9EE3509FAEF227E00C590
:2001EE00082FC508C5093EC50922E4F50AA88108E4F608B880FB22E4F520D201D200D20333
:20020E00D205C2B4E4F50EF50DF50CF50BE4F512F511F510F50F74FFF513E588543FF588A7
:20022E00E589540FF5894420F5897450F598E5874480F58774FAF58BF58DD28ED2AC22C052
:20024E00E0C0D0C083C082309839E50DB4FA028030502E050DE50DB50E0280044002F50E38
:20026E0090A000C0E0E50B2582F582E43583F583D0E0E599F0050BE50BB4FA004003750BEF
:20028E0000C298309948E511700DD200300235E4D5E0FDC2B4802DC20030011A300202D26D
:2002AE00B490A0FAC0E0E5102582F582E43583F583D0E0E0F59915110510E510B4FA00404F
:2002CE0003751000C299200105200002D299D082D083D0D0D0E0322278FB120048E6C0E0DE
:2002EE00B40A0B300308D204740D1581C0E0E511B4FA0280F950F7C2AC90A0FAC0E0E50FCD
:20030E002582F582E43583F583D0E0D0E0C0E0F00511050FE511B512004002F512E50FB4D5
:20032E00FA004003750F00300002D299D2ACD0E0300408C204740AC0E080B322E4F5F0786D
:20034E00FB120048F608A6F022E51364FF7038E50D6034300531C2AC90A000C0E0E50C2541
:20036E0082F582E43583F583D0E0E0D2ACB40A0302038574018010150D050CE50CB4FA0032
:20038E004003750C0080C875F00022E4A20192E0F51F70030203BAE51160030203A5E4A2F4
:2003AE000092E0F51FE51F70030203AC22C2AC7513FF7400F50CF50BC50DD2AC75F000221E
:2003CE0074FFC513B4FF2EE50D0060FBC2AC90A000C0E0E50C2582F582E43583F583D0E085
:2003EE00E0C0E0150D050CE50CB4FA004003750C00D2ACD0E030050BB40A030203D5B40D0F
:20040E0002740A75F000221203CEC0E0C0E0C0E01202E6D0E0D0E0D0E075F00022E5137506
:20042E00F0007BFF7C0012016E700302044374FFF5F002045378FB120048E60886F0F513A1
:20044E0018E60886F02278FB1200488682088683E06016C083C082C0E0C0E01202E6D0E045
:20046E00D0E0D082D083A380E722E4F5F078FB120048F608A6F02274BE75F054C0E0C0F066
:20048E00E52075F000C0E0C0F07402124FB0158115811581158174D975F054C0E0C0F0E57A
:2004AE000F75F000C0E0C0F0E510C0E0C0F0E51175F000C0E0C0F0E512C0E0C0F074057545
:2004CE00F000124FB07FF6120054740C75F055C0E0C0F0E50B75F000C0E0C0F0E50CC0E072
:2004EE00C0F0E50D75F000C0E0C0F0E50EC0E0C0F0740575F000124FB07FF6120054E4F5B1
:20050E000EF512227FFD7EFF1201EDE4F5F07F001201D1F0A3C5F0F0C5F078FB120048E6D1
:20052E000886F012013918F608A6F012012B45F06022181818860108860289828A831200B9
:20054E007589828A83E012008CC0E0C0F01250A91581158145F0700302061E7F001201D1CA
:20056E00E0A3F5F0E0C5F07B047C0012010B7F001201D1F0A3C5F0F0C5F078F912004886B6
:20058E000108860289828A8312007589828A83E012008CC0E0C0F01250B8158115817F0270
:2005AE001201D1F07F021201D1E012008C7B39120083120158600B7F021201D1E0C394308B
:2005CE00800B7F021201D1E0C39441240A75F0007F001201D112006E2BC5F03CC5F07F00DF
:2005EE001201D1F0A3C5F0F0C5F078F9120048860108860289828A83E0A3F5F0E0C5F01213
:20060E00012B89828A83F0A3C5F0F0C5F00205287F001201D1E0A3F5F0E0C5F07F03020187
:20062E00EB7FF17EFF1201ED7F021201DFE98AF0C0E0C0F0E4C0E0C0E0740A75F000C0E007
:20064E00C0F01250EA7FFA1200547F021201DFE98AF07F0C1201D1F0A3C5F0F0C5F0740902
:20066E007F0E1201D1F078FB120048860108860289828A8312007589828A83E012008CC032
:20068E00E0C0F01250701581158145F0602E78FB120048860108860289828A8312007589EF
:2006AE00828A83E012008CC0E0C0F01250A41581158145F060067F0E1201D1E07003020735
:2006CE003E7F0C1201D1E0A3F5F0E0C5F012012B7F0C1201D1F0A3C5F0F0C5F0120139F983
:2006EE00AAF0C001C00278F9120048860108860289828A8312007589828A83E0D083D082B1
:20070E00F018860108860289828A83E0A3F5F0E0C5F012012B89828A83F0A3C5F0F0C5F054
:20072E007F0E1201D1E0147F0E1201D1F00206747F021201DFE98AF0C0E0C0F012510D15BE
:20074E008115817F001201D1F0A3C5F0F0C5F07F0F0201EB7FFE7EFF1201EDE4F5F07F0066
:20076E001201D1F0A3C5F0F0C5F07F001201D1E0A3F5F0E0C5F012014C45F0601B78FB12A6
:20078E000048E60886F012013918F608A6F012012B7B007C0012016045F0700302080878CD
:2007AE00F7120048E60886F012012B18F608A6F0120139F9AAF089828A83E012008CC0E077
:2007CE00C0F008E60886F012012B18F608A6F0120139F9AAF089828A83E012008CFBACF0F9
:2007EE00D0F0D0E0C39BC5F09CC5F07F001201D1F0A3C5F0F0C5F00207787F001201D1E003
:20080E00A3F5F0E0C5F07F020201EB7FFF7EFF1201EDE47F001201D1F07F001201D1E07554
:20082E00F0007B107C0012018570120208887F001201D1E0047F001201D1F080DC78FB128C
:20084E000048E60886F07F001201D112006A2BC5F03400C5F0F9AAF07F001201D1E0C0019F
:20086E00C00279567AA412008C12007C89828A83E0F4D083D082F002083C740190A47AF0B5
:20088E007F010201EB7FFF7EFF1201EDE4F521E4F5F090A2BEF0A3C5F0F0C5F0E490A2BD6E
:2008AE00F074F475F0A1C0E0C0F0E4C0E0C0E074C975F000C0E0C0F01250EA7FFA1200543B
:2008CE00E4F5F090A389F0A3C5F0F0C5F074C075F0A2C0E0C0F0E4C0E0C0E074C975F00047
:2008EE00C0E0C0F01250EA7FFA120054E490A455F0748C75F0A3C0E0C0F0E4C0E0C0E07422
:20090E00C975F000C0E0C0F01250EA7FFA120054740190A47AF0E47F001201D1F07F001245
:20092E0001D1E075F0007B107C0012017F70120209997F001201D1E0047F001201D1F080B9
:20094E00DC7F001201D1E079567AA412008C12007C7F001201D1E0C001C00279687AA4127A
:20096E00008C12007C89828A83E0F412008CD083D08212006A120083120176700302099672
:20098E00E490A47AF002099902094090A47AE060030209DE745675F0A4C0E0C0F0E4C0E057
:2009AE00C0E0741275F000C0E0C0F01250EA7FFA120054745675F0A4C0E0C0F0747775F0B0
:2009CE0054C0E0C0F0125156158115811581158112175B1217F5746875F0A4C0E0C0F0126B
:2009EE000819158115817F010201EB12039978FB120048E60886F090A38BF0C209C2B490D0
:200A0E00A38BE075F000900A37020095E490A38BF0D208C202E490AC97F0020A4BC208D223
:200A2E0002E490AC97F0020A4B2B0A03002B0A02002B0A01001F0A000000001A0A227FFB1A
:200A4E007EFF1201ED78F9120048E60886F07F031201D1F0A3C5F0F0C5F008E60886F07F9E
:200A6E00011201D1F0A3C5F0F0C5F07F011201DFE98AF0C0E0C0F0740275F000C0E0C0F046
:200A8E0012051215811581158115817F001201D1F078FB120048E60886F0C0E0C0F074304F
:200AAE0075F000C0E0C0F07402C0E0C0F01250EA7FFA1200547F031201D112007589828A00
:200ACE0083E07003020B0F7F031201D11200757F001201D1E089828A8312006A2B7F001296
:200AEE0001D1F07F031201D1E0A3F5F0E0C5F012012B7F031201D1F0A3C5F0F0C5F0020A26
:200B0E00C37F001201D1E0F4047F001201D1F078FB12004886010886027F001201D1E075DA
:200B2E00F0007B047C00120119C001C00290547E12007512007C89828A83E0D083D082F009
:200B4E0078FB120048E60886F02401C5F03400C5F0F9AAF07F001201D1E0540FC001C002D7
:200B6E0090547E12007512008C12007C89828A83E0D083D082F07F001201D1E012008C5490
:200B8E00FFC5F05400C5F07F050201EB90A455E06003020C40748C75F0A3C0E0C0F0E4C002
:200BAE00E0C0E074C975F000C0E0C0F01250EA7FFA12005490A38BE075F0007B007C00127E
:200BCE00018D7003020C2C798C7AA3742489828A83F0E4A20992E0F51F748C75F0A3C0E04D
:200BEE00C0F0E51F6007745075F0558005745475F055C0E0C0F01251461581158115811577
:200C0E0081748C75F0A3C0E0C0F0745675F0A4C0E0C0F01251461581158115811581748CC9
:200C2E0075F0A3C0E0C0F01251841581158190A455F078FB120048E60886F07B0A7C00127E
:200C4E00016E700C18E60886F07BFF7C0012016E45F07003020CD1E4A20992E0F51F700399
:200C6E00020C94748C75F0A3C0E0C0F0748C75F0A32401C5F03400C0F0C0E0120A4C158108
:200C8E00158115811581748C75F0A3C0E0C0F01204541581158178FB120048E60886F07BEA
:200CAE000A7C0012016E7003020CC9740A75F000C0E0C0F01202E615811581E490A455F01F
:200CCE00020CFD748C75F0A390A45512006A2BC5F03400C5F0F9AAF078FB120048E6088651
:200CEE00F089828A83F090A455E00490A455F02278FB120048860108860289828A83E0709A
:200D0E0003020D3F18860108860289828A83E012008CC0E0C0F0120B9A1581158178FB12F7
:200D2E000048E60886F012012B18F608A6F0020CFE227FFA7EFF1201EDE4F5F07F0212018E
:200D4E00D1F0A3C5F0F0C5F078FB120048E60886F07F001201D1F0A3C5F0F0C5F0E47F04DF
:200D6E001201D1F07F041201D1E075F0007B027C0012017F7003020FC07F041201D1E0755A
:200D8E00F000900F96020095C2097F001201D1E0A3F5F0E0C5F012012B7F001201D1F0A32A
:200DAE00C5F0F0C5F0120139F9AAF089828A83E012008C900F0D0200957F001201D112009E
:200DCE007589828A83E012008C7B2012008312016E7003020DEF74017F041201D1F0020DFD
:200DEE00F774037F041201D1F0020F1978FB120048E60886F0C0E0C0F018E60886F02401D4
:200E0E00C5F03400C0F0C0E0120A4C15811581158115817F051201D1F07F051201D1E070BB
:200E2E0003020EAD74037F041201D1F0742F75F075C0E0C0F090A2BEE0A3F5F0E0C5F0124A
:200E4E00012B90A2BEF0A3C5F0F0C0F0C0E01251CB158115811581158190A2BEF0A3C5F022
:200E6E00F0C5F090A38BE075F0007B027C0012016E7003020EAA745675F055C0E0C0F07FC2
:200E8E00051201D1E075F000C0E0C0F0740275F000124FB01581158115811581020EFF7FF4
:200EAE00001201D1E0A3F5F0E0C5F02402C5F03400C5F07F001201D1F0A3C5F0F0C5F07FB0
:200ECE00001201D112007589828A83E012008C7B2012008312016E7003020EF774017F04E0
:200EEE001201D1F0D209020EFF74037F041201D1F0020F1974037F041201D1F0020F19FA3C
:200F0E000D2300C70D21000000020F020FA2745675F0A4C0E0C0F07F001201D1E0A3F5F0EC
:200F2E00E0C0F0C0E0745675F0A4C0E0C0F012518415811581C0E0C0F01207627FFA1200E7
:200F4E005445F07003020F6174037F041201D1F0020F9374027F041201D1F0745675F0A403
:200F6E00C0E0C0F0125184158115817F001201D112006E2BC5F03CC5F07F021201D1F0A354
:200F8E00C5F0F0C5F0020FA21C0F0100960D00000000A20F7F001201D1E0A3F5F0E0C5F056
:200FAE0012012B7F001201D1F0A3C5F0F0C5F0020D727F021201D1E0A3F5F0E0C5F07F062D
:200FCE000201EB7FFD7EFF1201EDE4F5F07F011201D1F0A3C5F0F0C5F012035745F07003EE
:200FEE000212741203CE7F001201D1F0E4A20892E0F51F700302101A7F001201D1E012001D
:20100E008CC0E0C0F01202E61581158190A2BDE0600302104274F475F0A1C0E0C0F0E4C0D8
:20102E00E0C0E074C975F000C0E0C0F01250EA7FFA1200547F001201D1E012008C9010BACA
:20104E0002009590A2BDE0700302107390A2BDE01490A2BDF079F47AA112008C12007CE4CA
:20106E0089828A83F00210C60210C674F475F0A190A2BD12006A2BC5F03400C5F0F9AAF075
:20108E007F001201D1E089828A83F090A2BDE00490A2BDF075F0007BC87C00120195700306
:2010AE000210B774C790A2BDF00210C676100A0051100800000079107F001201D1E0120090
:2010CE008C7B0A12008312016E700302127490A38BE075F00090125B02009579F47AA18938
:2010EE00828A83E012008C7B2A120083120176700302111374F475F0A17F011201D1F0A314
:20110E00C5F0F0C5F002126F74F475F0A1C0E0C0F0120D40158115817F011201D1F0A3C5DF
:20112E00F0F0C5F002126F90A2BDE070030211B279F47AA189828A83E012008C9011A2021F
:20114E0000950211B2746D75F055C0E0C0F01204541581158174F475F0A1C0E0C0F01204D2
:20116E005415811581746F75F055C0E0C0F01204541581158174F475F0A1C0E0C0F0120D81
:20118E0040158115817F011201D1F0A3C5F0F0C5F00211B250112D0050112A005011240021
:2011AE000000531102126F90A2BDE0700302124579F47AA189828A83E012008C90123502A8
:2011CE00009502124574F475F0A1C0E0C0F0120D40158115817F011201D1F0A3C5F0F0C569
:2011EE00F07F011201D1E0A3F5F0E0C5F045F07003021232747175F055C0E0C0F012045449
:20120E0015811581745675F0A4C0E0C0F012045415811581747575F055C0E0C0F01204547E
:20122E0015811581021245D0112D00D0112A00D01124000000D31102126F740175F000C0FC
:20124E00E0C0F01209F91581158102126FB51103003511020016110100E9100000000048B3
:20126E0012E490A2BDF07F011201D1E0A3F5F0E0C5F07F030201EB90A38BE075F0007B003C
:20128E007C0012016E700E90A38BE075F0007B027C0012016E45F070030212BE78FB120049
:2012AE0048E60886F0C0E0C0F0120CFE158115812290A38BE075F0007B007C0012016E70CF
:2012CE00030212F2745675F0A4C0E0C0F012045415811581747975F055C0E0C0F0120454DD
:2012EE0015811581227FFD7EFF1201ED78FB120048E60886F02401C5F03400C5F0F9AAF012
:20130E0089828A83E012008C7B3D12008312016E700302144E18E60886F02402C5F03400F9
:20132E00C5F07F001201D1F0A3C5F0F0C5F07F001201D1E0A3F5F0E0C0F0C0E012518415A3
:20134E008115817B017C00120168700302143B745675F0A4C0E0C0F0E4C0E0C0E0741275EF
:20136E00F000C0E0C0F01250EA7FFA120054E47F021201D1F07F021201D1E075F0007B1086
:20138E007C0012017F600D7F001201D112007589828A83E070120213F87F021201D1E0040A
:2013AE007F021201D1F080CD7F021201D1E079567AA412008C12007C7F001201D1E0A3F544
:2013CE00F0E0C5F012012B7F001201D1F0A3C5F0F0C5F0120139C001C002F9AAF089828AF5
:2013EE0083E0D083D082F00213A7745675F0A4C0E0C0F0745675F0A4C0E0C0F012518415E9
:20140E00811581D004D0032BC5F03CC5F0F9AAF0742089828A83F012175B746875F0A4C0D7
:20142E00E0C0F01208191581158102144B747B75F055C0E0C0F012128515811581021499D1
:20144E0012175B746875F0A4C0E0C0F01208191581158174C075F0A2C0E0C0F0749575F06D
:20146E0055C0E0C0F0745675F0A4C0E0C0F0740375F000124FC17FFA12005474C075F0A27E
:20148E00C0E0C0F0120CFE158115817F030201EB78FB120048E60886F018F608A6F074C025
:2014AE0075F0A2C0E0C0F074A875F055C0E0C0F0745675F0A4C0E0C0F0740375F000124F41
:2014CE00C17FFA12005474C075F0A2C0E0C0F0120CFE15811581788018E660FC881F74C05E
:2014EE0075F0A2C0E0C0F074B975F055C0E0C0F0E51F75F000C0E0C0F0747FC0E0C0F074E0
:20150E000475F000124FC17FF812005474C075F0A2C0E0C0F0120CFE158115812278FB12DB
:20152E000048E60886F018F608A6F074C075F0A2C0E0C0F074D375F055C0E0C0F0E50A7505
:20154E00F000C0E0C0F090A2BEE0A3F5F0E0C0F0C0E0740475F000124FC17FF81200547465
:20156E00C075F0A2C0E0C0F0120CFE15811581E4F50AE4F5F090A2BEF0A3C5F0F0C5F02253
:20158E007FFE7EFF1201ED78FB120048E60886F02401C5F03400C5F07F001201D1F0A3C594
:2015AE00F0F0C5F07F001201D112007589828A83E012008CC0E0C0F01250A4158115814541
:2015CE00F070030215F07F001201D1E0A3F5F0E0C0F0C0E012510D1581158190AC97F00237
:2015EE00162A74C075F0A2C0E0C0F0740275F056C0E0C0F090AC97E075F000C0E0C0F074B5
:20160E000375F000124FC17FFA12005474C075F0A2C0E0C0F0120CFE158115817F020201FC
:20162E00EB7FFE7EFF1201ED78FB120048E60886F02401C5F03400C5F07F001201D1F0A3CD
:20164E00C5F0F0C5F07F001201D112007589828A83E012008C9016FE02009574C075F0A22C
:20166E00C0E0C0F0741675F056C0E0C0F090A38BE075F000C0E0C0F0740375F000124FC126
:20168E007FFA12005474C075F0A2C0E0C0F0120CFE158115810217067F001201D112007581
:2016AE0089828A83E012008CC0E0C0F01250A41581158145F070030216EB7F001201D1E016
:2016CE00A3F5F0E0C0F0C0E012510D15811581C0E0C0F01209F9158115810216FB742675F6
:2016EE00F056C0E0C0F012128515811581021706691600000000A6167F020201EB90A38BEA
:20170E00E075F0007B007C0012016E700302175A74C075F0A2C0E0C0F0743E75F056C0E080
:20172E00C0F078F7120048E60886F0C0E0C0F0740375F000124FC17FFA12005474C075F0F8
:20174E00A2C0E0C0F012128515811581227FFD7EFF1201EDE590F4540E12008C7B011200A2
:20176E00831201197F001201D1F07F001201D1E044307F011201D1F0745675F0A4C0E0C01B
:20178E00F0125184158115817F021201D1F07F021201D1E075F0007B027C00120195700325
:2017AE000217D27F021201D1E0C3940279567AA412008C12007C7F011201D1E089828A831D
:2017CE00F00217E7E4F5F079567AA412007C7F011201D1E089828A83F07F001201D1E01226
:2017EE00008C7F030201EBD290A290B3E492E0F51FE51F7003021815E4C0E0C0E01209F950
:20180E0015811581021825740175F000C0E0C0F01209F915811581227FF87EFF1201ED7857
:20182E00FB120048E60886F07F021201D1F0A3C5F0F0C5F07F001201D1F0A3C5F0F0C5F03F
:20184E007F001201D112007589828A83E070030219007F001201D112007589828A83E01216
:20186E00008C7B2012008312016E700302189B7F001201D1E0A3F5F0E0C5F012012B7F00D8
:20188E001201D1F0A3C5F0F0C5F00218FD7F021201D1120075C001C0027F001201D112006E
:2018AE007589828A83E012008CC0E0C0F01250B815811581D083D082F07F001201D1E0A3FE
:2018CE00F5F0E0C5F012012B7F001201D1F0A3C5F0F0C5F07F021201D1E0A3F5F0E0C5F090
:2018EE0012012B7F021201D1F0A3C5F0F0C5F002184E7F021201D1120075E489828A83F00A
:20190E0078FB120048E60886F02401C5F03400C5F07F001201D1F0A3C5F0F0C5F0188601D6
:20192E0008860289828A83E012008C901DBA02009578FB120048E60886F0C0E0C0F01212D0
:20194E00F315811581021DEA021DEA12149E74C075F0A2C0E0C0F0745975F056C0E0C0F021
:20196E00E51675F000C0E0C0F07403124FC17FFA12005474C075F0A2C0E0C0F0120CFE1575
:20198E00811581021DEA78FB120048E60886F0C0E0C0F012152B15811581021DEA78FB128C
:2019AE000048E60886F0C0E0C0F012158E15811581021DEA78FB120048E60886F0C0E0C0A2
:2019CE00F012162F15811581021DEA7F001201D112007589828A83E012008C7B41120083AC
:2019EE0012016E60277F001201D1E0A3F5F0E0C5F02401C5F03400C5F0F9AAF089828A8303
:201A0E00E012008C7B3112008312015845F07003021AC87F001201D1E0A3F5F0E0C5F01290
:201A2E00012B7F001201D1F0A3C5F0F0C5F07F001201D112007589828A83E012008C901AF2
:201A4E00B5020095E4C0E0C0E0124B8415811581740A75F000C0E0C0F0120B9A15811581E5
:201A6E00740175F000C0E0C0F0124B8415811581021AC57F001201D112007589828A83E05E
:201A8E00C3943012008CC0E0C0F0124B8415811581021AC5746575F056C0E0C0F012128548
:201AAE0015811581021AC5811A3100811A3000521A00000000A21A021C197F001201D112A0
:201ACE00007589828A83E07003021C197F001201DFE98AF0C0E0C0F07F041201DFE98AF0E5
:201AEE00C0E0C0F07F061201DFE98AF0C0E0C0F01239F67FFA12005445F06003021C197FF0
:201B0E00041201D1E0A3F5F0E0C5F05400C5F0540FC5F07B087C00120119901BC202009582
:201B2E007F041201D1E0A3F5F0E0C5F05400C5F05440C5F045F07003021B6E7F041201D147
:201B4E00E0A3F5F0E0C0F0C0E0742775F054C0E0C0F01249BC1581158115811581021B951A
:201B6E007F041201D1E0A3F5F0E0C0F0C0E07F061201D1E0A3F5F0E0C0F0C0E0123DA31550
:201B8E0081158115811581021BCE7F041201D1E0A3F5F0E0C0F0C0E07F061201D1E0A3F529
:201BAE00F0E0C0F0C0E0123DA31581158115811581021BCE2E1B06002E1B02000000981B75
:201BCE007F001201D112007589828A83E012008C7B2C12008312016E7003021C167F001282
:201BEE0001D1E0A3F5F0E0C5F012012B7F001201D1F0A3C5F0F0C5F0742C75F000C0E0C015
:201C0E00F0120B9A15811581021AC8740A75F000C0E0C0F0120B9A15811581021DEA7F0061
:201C2E001201D1E0A3F5F0E0C0F0C0E0747C75F056C0E0C0F0125212158115811581158151
:201C4E0045F07003021C68748175F056C0E0C0F012128515811581021C70120399C2AF02C4
:201C6E000000021DEA7F001201D112007589828A83E07003021CEA7F001201DFE98AF0C05C
:201C8E00E0C0F07F041201DFE98AF0C0E0C0F012365F158115811581158145F06003021CC9
:201CAE00EA7F001201D112007589828A83E012008C7B2C12008312016E7003021CE77F00F8
:201CCE001201D1E0A3F5F0E0C5F012012B7F001201D1F0A3C5F0F0C5F0021C73021DEA02EB
:201CEE001DEA749675F056C0E0C0F0120CFE1581158174CB75F056C0E0C0F0120CFE158176
:201D0E00158174F875F056C0E0C0F0120CFE15811581743775F057C0E0C0F0120CFE1581F7
:201D2E001581746175F057C0E0C0F0120CFE15811581748F75F057C0E0C0F0120CFE158115
:201D4E00158174AF75F057C0E0C0F0120CFE1581158174CB75F057C0E0C0F0120CFE15816B
:201D6E001581740075F058C0E0C0F0120CFE15811581742175F058C0E0C0F0120CFE1581A2
:201D8E001581744075F058C0E0C0F0120CFE15811581021DEA78FB120048E60886F0C0E0BC
:201DAE00C0F012170B15811581021DEAF01C3F00ED1C0000731C53002C1C5200D9195100E9
:201DCE00C2194E00AB194C009419450059194400561943003F1941000000A31D7F0802017F
:201DEE00EBE4F522E4F516F518740E75F0DCF51485F015E58854CFF588E58954F0F589441C
:201E0E0001F589E4F58AF58CD2A9D28C22C0E0C0D0C28C85148A85158CD28C05170516E515
:201E2E0016B464004006D217249CF516301603851618D0D0D0E032227FFF7EFF1201EDE5EC
:201E4E00167F001201D1F07F001201D1E075F000AB167C0012016E6003021E5578FB120048
:201E6E0048E60886F012013918F608A6F012012B45F06003021E4D7F010201EB78FB12007A
:201E8E0048E60886F045F07003021EB875F02ED5F0FD78FB120048E60886F012013918F628
:201EAE0008A6F045F06003021E9A2290AC97E054207003021F3074C075F0A2C0E0C0F07418
:201ECE005C75F058C0E0C0F078F7120048E60886F0C0E0C0F078F1120048E60886F0C333F1
:201EEE00C5F033C5F079077A5412007C89828A83E0A3F5F0E0C5F078F312004826C5F0089E
:201F0E0036C0F0C0E0740475F000124FC17FF812005474C075F0A2C0E0C0F0121285158187
:201F2E00158178F7120048E60886F0C333C5F033C5F079077A5412007C89828A83E0A3F5D1
:201F4E00F0E0C5F078F912004826C5F00836C0F0C0E008E60886F0C0E0C0F012526915819B
:201F6E0015811581158178F7120048E60886F07B207C001200BEC0E0C0F008E60886F0C3FE
:201F8E0033C5F033C5F0D004D0032BC5F03CC5F0797E7AA412007C89828A83E0A3F5F0E0E8
:201FAE00C5F05410C5F05400C5F045F0700302200478F7120048E60886F07B207C00120018
:201FCE00BEC0E0C0F008E60886F0C333C5F033C5F0D004D0032BC5F03CC5F0797E7AA81243
:201FEE00007C78FB120048E60886F089828A83F0A3C5F0F0C5F0227FFD7EFF1201ED78F995
:20200E00120048E60886F07B207C001200BEC0E0C0F008E60886F0C333C5F033C5F0D004EA
:20202E00D0032BC5F03CC5F0797E7AA412007C89828A83E0A3F5F0E0C5F05410C5F05400C9
:20204E00C5F045F070030220AA78F9120048E60886F07B207C001200BEC0E0C0F008E608ED
:20206E0086F0C333C5F033C5F0D004D0032BC5F03CC5F0797E7AA812007C89828A83E0A38F
:20208E00F5F0E0C5F07F001201D1F0A3C5F0F0C5F074017F021201D1F00220F478F9120005
:2020AE0048E60886F0C333C5F033C5F079077A5412007C89828A83E0A3F5F0E0C5F078FB6F
:2020CE0012004826C5F00836C0F0C0E0125248158115817F001201D1F0A3C5F0F0C5F0E423
:2020EE007F021201D1F090AC97E05420700302218474C075F0A2C0E0C0F0747875F058C048
:20210E00E0C0F07F001201D1E0A3F5F0E0C0F0C0E078F3120048E60886F0C333C5F033C55A
:20212E00F079077A5412007C89828A83E0A3F5F0E0C5F078F512004826C5F00836C0F0C060
:20214E00E07F021201D1E06007749875F0588005749E75F058C0E0C0F0740575F000124F39
:20216E00C17FF612005474C075F0A2C0E0C0F0120CFE158115817F001201D1E0A3F5F0E037
:20218E00C5F07F030201EB7FFF7EFF1201EDE4F5F090A47BF0A3C5F0F0C5F0741090A47D77
:2021AE00F0749F75F058C0E0C0F012128515811581747E75F0A4C0E0C0F0E4C0E0C0E0E4D9
:2021CE0075F001C0E0C0F01250EA7FFA120054747E75F0A5C0E0C0F0E4C0E0C0E0E475F057
:2021EE0001C0E0C0F01250EA7FFA120054747E75F0A6C0E0C0F0E4C0E0C0E0E475F001C0DA
:20220E00E0C0F01250EA7FFA120054747E75F0A7C0E0C0F0E4C0E0C0E0E475F001C0E0C0D9
:20222E00F01250EA7FFA120054747E75F0A8C0E0C0F0E4C0E0C0E0E475F001C0E0C0F01256
:20224E0050EA7FFA120054747E75F0A9C0E0C0F0E4C0E0C0E0E475F001C0E0C0F01250EAFD
:20226E007FFA120054747E75F0AAC0E0C0F0E4C0E0C0E0E475F001C0E0C0F01250EA7FFA9D
:20228E00120054E47F001201D1F07F001201D1E075F0007B087C0012017F70120223C47F70
:2022AE00001201D1E0047F001201D1F080DC74C075F0A2C0E0C0F074C075F058C0E0C0F0CD
:2022CE007F001201D1E075F000C333C5F033C5F079F77A5312007C89828A83E0A3F5F0E08A
:2022EE00C0F0C0E0740375F000124FC17FFA12005474C075F0A2C0E0C0F0121285158115C4
:20230E00817F001201D1E075F00090238D0200957F001201D1E075F000C0E0C0F01223FC86
:20232E00158115810223B17F001201D1E075F000C0E0C0F0122656158115810223B17F0086
:20234E001201D1E075F000C0E0C0F01227F2158115810223B17F001201D1E075F000C0E081
:20236E00C0F0122C8C158115810223B174C975F058C0E0C0F0121285158115810223B1637B
:20238E00230700632303004C2306004C23020035230500352301001E2304001E230000005A
:2023AE00007A2374DE75F058C0E0C0F0121285158115810222AD744075F000797E7AA4122D
:2023CE00007C89828A83E0A3F5F0E0C5F05401C5F05400C5F045F070030223F3D288D2A8B7
:2023EE00D2160223F7C288C2A87F010201EB7FFD7EFF1201EDE4F5F07F001201D1F0A3C52C
:20240E00F0F0C5F0740275F000C0E0C0F0121E461581158178FB120048E60886F09026392C
:20242E00020095E47F021201D1F078FB120048E60886F0C333C5F033C5F079077A5412009A
:20244E007C89828A83E0A3F5F0E0C0F0C0E0740775F000C0E0C0F012526915811581158183
:20246E001581C2AF75F000E4A2B33400D5F0F9D2AFF51FE51F700302257078FB120048E661
:20248E000886F07B207C001200BE2400C5F03400C5F0797E7AA412007C89828A83E0A3F5D4
:2024AE00F0E0C5F04401C5F04400C5F089828A83F0A3C5F0F0C5F074C075F0A2C0E0C0F006
:2024CE0074E075F058C0E0C0F01251561581158115811581E51F75F0007B097C0012017F81
:2024EE00700302255078FB120048E60886F07B207C001200BE2400C5F03400C5F0797E7A99
:20250E00A412007C89828A83E0A3F5F0E0C5F04406C5F04400C5F089828A83F0A3C5F0F01E
:20252E00C5F074C075F0A2C0E0C0F074E975F058C0E0C0F0125146158115811581158102E0
:20254E00256D74C075F0A2C0E0C0F074F175F058C0E0C0F0125146158115811581158102DB
:20256E00259E74C075F0A2C0E0C0F074F975F058C0E0C0F012515615811581158115817400
:20258E000175F0007F001201D1F0A3C5F0F0C5F074C075F0A2C0E0C0F01212851581158117
:2025AE0074C075F0A2C0E0C0F0740775F059C0E0C0F0E51F75F000C0E0C0F07403124FC1A7
:2025CE007FFA12005474C075F0A2C0E0C0F01212851581158102264578FB120048E6088600
:2025EE00F07B207C001200BE2400C5F03400C5F0797E7AA412007C89828A83E0A3F5F0E031
:20260E00C5F04401C5F04400C5F089828A83F0A3C5F0F0C5F0741675F059C0E0C0F0121243
:20262E008515811581022645022645E625040031240000000036267F001201D1E0A3F5F076
:20264E00E0C5F07F030201EB7FFD7EFF1201EDE4F5F07F001201D1F0A3C5F0F0C5F0E47FF2
:20266E00021201D1F078FB120048E60886F0C333C5F033C5F079177A5412007C7F02120132
:20268E00D1E075F00089828A8312006E12017F70120227077F021201D1E0047F021201D18C
:2026AE00F080C278FB120048E60886F07B207C001200BEC0E0C0F07F021201D1E075F000C8
:2026CE00C333C5F033C5F0D004D0032BC5F03CC5F0797E7AA412007C89828A83E0A3F5F0BE
:2026EE00E0C5F04410C5F04400C5F089828A83F0A3C5F0F0C5F00226A278FB120048E608AB
:20270E0086F09027D502009578FB120048E60886F07B207C001200BE2400C5F03400C5F038
:20272E00797E7AA412007C89828A83E0A3F5F0E0C5F04401C5F04400C5F089828A83F0A335
:20274E00C5F0F0C5F0742575F059C0E0C0F012128515811581E47F021201D1F078FB1200D7
:20276E0048E60886F0C333C5F033C5F079177A5412007C7F021201D1E075F00089828A835E
:20278E0012006E12017F70120227D27F021201D1E0047F021201D1F080C278FB120048E609
:2027AE000886F0C0E0C0F07F021201D1E075F000C0E0C0F0E4C0E0C0E0121EB97FFA1200AB
:2027CE00540227990227E116270500162701000000E1277F001201D1E0A3F5F0E0C5F07F64
:2027EE00030201EB7FFD7EFF1201EDE4F5F07F001201D1F0A3C5F0F0C5F0E4F5F07F00126E
:20280E0001D1F0A3C5F0F0C5F078FB120048E60886F0C333C5F033C5F079077A5412007C4B
:20282E0089828A83E0A3F5F0E0C5F0240DC5F03400C0F0C0E0740775F000C0E0C0F0125277
:20284E0069158115811581158178FB120048E60886F0C333C5F033C5F079077A5412007C09
:20286E0089828A83E0A3F5F0E0C0F0C0E0125248158115817F021201D1F078FB120048E6BA
:20288E000886F0C333C5F033C5F079077A5412007C89828A83E0A3F5F0E0C0F0C0E0740613
:2028AE0075F000C0E0C0F0125269158115811581158178FB120048E60886F0C333C5F03321
:2028CE00C5F079077A5412007C89828A83E0A3F5F0E0C0F0C0E012524815811581540FC5A9
:2028EE00F05400C5F07B067C001201767003022910740175F0007F001201D1F0A3C5F0F028
:20290E00C5F078FB120048E60886F0C333C5F033C5F079077A5412007C89828A83E0A3F5C4
:20292E00F0E0C0F0C0E0740975F000C0E0C0F0125269158115811581158178FB120048E65F
:20294E000886F0C333C5F033C5F079077A5412007C89828A83E0A3F5F0E0C0F0C0E0125268
:20296E004815811581540FC5F05400C5F07B097C001201767003022998740175F0007F009C
:20298E001201D1F0A3C5F0F0C5F078FB120048E60886F0C333C5F033C5F079077A54120034
:2029AE007C89828A83E0A3F5F0E0C0F0C0E07F021201D1E075F000C0E0C0F0125269158180
:2029CE0015811581158178FB120048E60886F0C333C5F033C5F079077A5412007C89828AF2
:2029EE0083E0A3F5F0E0C5F0240DC5F03400C0F0C0E0740675F000C0E0C0F012526915814D
:202A0E001581158115817F001201D1E0A3F5F0E0C5F045F07003022A3A744975F059C0E05D
:202A2E00C0F012128515811581022C7B745775F059C0E0C0F01212851581158178FB120027
:202A4E0048E60886F07B207C001200BE2400C5F03400C5F0797E7AA412007C89828A83E078
:202A6E00A3F5F0E0C5F04401C5F04400C5F089828A83F0A3C5F0F0C5F078FB120048E60878
:202A8E0086F0902C6F02009578FB120048E60886F0C333C5F033C5F079077A5412007C89C7
:202AAE00828A83E0A3F5F0E0C5F0240EC5F03400C0F0C0E0740475F000C0E0C0F012526917
:202ACE001581158115811581746175F059C0E0C0F01212851581158178FB120048E6088697
:202AEE00F0C333C5F033C5F079077A5412007C89828A83E0A3F5F0E0C5F0240FC5F0340038
:202B0E00C0F0C0E012524815811581540FC5F05400C5F07F021201D1F07F021201D1E05470
:202B2E000412008C12014C45F070087F021201D1E054017003022C1678FB120048E6088647
:202B4E00F0C333C5F033C5F079077A5412007C89828A83E0A3F5F0E0C5F0240FC5F03400D7
:202B6E00C0F0C0E0740175F000C0E0C0F0125269158115811581158178FB120048E6088667
:202B8E00F0C333C5F033C5F079077A5412007C89828A83E0A3F5F0E0C5F0240FC5F0340097
:202BAE00C0F0C0E0740575F000C0E0C0F0125269158115811581158178FB120048E6088623
:202BCE00F0C333C5F033C5F079077A5412007C89828A83E0A3F5F0E0C5F0240FC5F0340057
:202BEE00C0F0C0E0740475F000C0E0C0F01252691581158115811581746F75F059C0E0C024
:202C0E00F012128515811581022C7B78FB120048E60886F0C333C5F033C5F079077A541214
:202C2E00007C89828A83E0A3F5F0E0C5F0240EC5F03400C0F0C0E0740175F000C0E0C0F060
:202C4E001252691581158115811581748575F059C0E0C0F012128515811581022C7B022C8E
:202C6E007B192C0600962A020000006C2C7F001201D1E0A3F5F0E0C5F07F030201EB7FFED9
:202C8E007EFF1201EDE4F5F07F001201D1F0A3C5F0F0C5F078FB120048E60886F07B207C48
:202CAE00001200BE2400C5F03400C5F0797E7AA412007C89828A83E0A3F5F0E0C5F0440177
:202CCE00C5F04400C5F089828A83F0A3C5F0F0C5F078FB120048E60886F07B207C001200D9
:202CEE00BE2404C5F03400C5F0797E7AA412007C89828A83E0A3F5F0E0C5F04400C5F0444D
:202D0E0002C5F089828A83F0A3C5F0F0C5F078FB120048E60886F07B207C001200BE2406A7
:202D2E00C5F03400C5F0797E7AA412007C89828A83E0A3F5F0E0C5F04410C5F04400C5F02D
:202D4E0089828A83F0A3C5F0F0C5F078FB120048E60886F0C0E0C0F0740375F000C0E0C0A3
:202D6E00F07492C0E0C0F0121EB97FFA12005474A075F059C0E0C0F0121285158115817FC1
:202D8E00001201D1E0A3F5F0E0C5F07F020201EBC0E0C0D0C28C85148A85158CD28CE516B5
:202DAE00600DB46304D28D8006751600751800D0D0D0E032227FFE7EFF1201ED78FB12005D
:202DCE0048E60886F07B007C0012016E7003022E5CE4A2B392E0F51F7003022E5C7401751A
:202DEE00F00018F608A6F0E51F75F00045F0600690AC97E054017003022E5C74C075F0A2E3
:202E0E00C0E0C0F074D375F059C0E0C0F078F3120048E60886F0C333C5F033C5F079F77A59
:202E2E005312007C89828A83E0A3F5F0E0C0F0C0E0740375F000124FC17FFA12005474C0E2
:202E4E0075F0A2C0E0C0F01212851581158178F7120048E60886F0C333C5F033C5F07907F8
:202E6E007A5412007C89828A83E0A3F5F0E0C5F078F912004826C5F00836C0F0C0E0E4C0FB
:202E8E00E0C0E0125269158115811581158175F046D5F0FDE4F51F7003022EBD74FFF5F062
:202EAE007F001201D1F0A3C5F0F0C5F0022FCA78F7120048E60886F07B207C001200BE2481
:202ECE0000C5F03400C5F0797E7AA412007C89828A83E0A3F5F0E0C5F05404C5F05400C568
:202EEE00F045F07003022F9378F7120048E60886F0C333C5F033C5F079077A5412007C8943
:202F0E00828A83E0A3F5F0E0C0F0C0E01252481581158154FFC5F05400C5F07B027C001288
:202F2E00010B7F001201D1F0A3C5F0F0C5F078F7120048E60886F0C333C5F033C5F07907E7
:202F4E007A5412007C89828A83E0A3F5F0E0C0F0C0E01252481581158154FFC5F05400C55E
:202F6E00F07B067C001201197F001201D112006E4BC5F04CC5F07F001201D1F0A3C5F0F0AB
:202F8E00C5F0022FCA78F7120048E60886F0C333C5F033C5F079077A5412007C89828A83BF
:202FAE00E0A3F5F0E0C0F0C0E0125248158115817F001201D1F0A3C5F0F0C5F0E51F75F0DA
:202FCE000045F0600690AC97E05401700302304C74C075F0A2C0E0C0F074F775F059C0E0FB
:202FEE00C0F078F3120048E60886F0C333C5F033C5F079F77A5312007C89828A83E0A3F5FC
:20300E00F0E0C0F0C0E078F3120048E60886F0C0E0C0F07F001201D1E0A3F5F0E0C0F0C0EE
:20302E00E0740575F000124FC17FF612005474C075F0A2C0E0C0F0121285158115817F00E8
:20304E001201D1E0A3F5F0E0C5F07F020201EB7FF87EFF1201EDE47F061201D1F07F05124B
:20306E0001D1F0E475F0E07F001201D1F0A3C5F0F0C5F0747E75F0ABC0E0C0F0E4C0E0C071
:20308E00E074C975F000C0E0C0F01250EA7FFA120054747E75F0AB7F021201D1F0A3C5F076
:2030AE00F0C5F078FB120048860108860289828A8312007589828A83E012008CC0E0C0F0F4
:2030CE001250701581158145F0602478FB120048860108860289828A8312007589828A8390
:2030EE00E012008CC0E0C0F012508E1581158145F070030231787F021201D1E0A3F5F0E0D8
:20310E00C5F012012B7F021201D1F0A3C5F0F0C5F0120139F9AAF0C001C00278F91200482F
:20312E00860108860289828A8312007589828A83E012008CC0E0C0F01250B815811581D0CF
:20314E0083D082F078FB120048860108860289828A83E0A3F5F0E0C5F012012B89828A834D
:20316E00F0A3C5F0F0C5F00230B1E47F041201D1F07F041201D1E075F0007B087C00120178
:20318E007F70120231E57F041201D1E0047F041201D1F080DC747E75F0ABC0E0C0F07F0435
:2031AE001201D1E075F000C333C5F033C5F079F77A5312007C89828A83E0A3F5F0E0C0F06A
:2031CE00C0E0125212158115811581158145F070030231E50231947F041201D1E075F00040
:2031EE007B087C0012016E700302323574C075F0A2C0E0C0F0740675F05AC0E0C0F0747E5F
:20320E0075F0ABC0E0C0F0740375F000124FC17FFA12005474C075F0A2C0E0C0F01212852F
:20322E00158115810235FD7F001201D1E0A3F5F0E0C5F054FFC5F0547FC5F07F001201D1CD
:20324E00F0A3C5F0F0C5F090AC97E05420700302329874C075F0A2C0E0C0F0742075F05A2F
:20326E00C0E0C0F0747E75F0ABC0E0C0F0740375F000124FC17FFA12005474C075F0A2C0C6
:20328E00E0C0F0120CFE1581158178FB120048860108860289828A8312007589828A83E0CD
:2032AE0012008C7B2E12008312016E700302340E18860108860289828A83E0A3F5F0E0C598
:2032CE00F012012B89828A83F0A3C5F0F0C5F018E60886F0C0E0C0F012062F158115817FEF
:2032EE00071201D1F07F041201D1E075F000C333C5F033C5F079177A5412007C7F07120121
:20330E00D1E075F00089828A8312006E12017F70030233987F071201D1E07F051201D1F07D
:20332E007F001201D1E0A3F5F0E0C5F054FFC5F054BFC5F07F001201D1F0A3C5F0F0C5F0FF
:20334E0090AC97E05420700302339574C075F0A2C0E0C0F0742B75F05AC0E0C0F07F07122A
:20336E0001D1E075F000C0E0C0F0740375F000124FC17FFA12005474C075F0A2C0E0C0F070
:20338E00120CFE1581158102340BE475F0807F001201D1F0A3C5F0F0C5F074C075F0A2C082
:2033AE00E0C0F0743A75F05AC0E0C0F07F041201D1E075F000C333C5F033C5F079F77A5336
:2033CE0012007C89828A83E0A3F5F0E0C0F0C0E07F071201D1E075F000C0E0C0F0740475B5
:2033EE00F000124FC17FF812005474C075F0A2C0E0C0F0121285158115810235FD023429DD
:20340E0090AC97E054207003023429745775F05AC0E0C0F0120CFE1581158178FB120048B6
:20342E00860108860289828A8312007589828A83E012008C7B2E12008312016E70030235C9
:20344E00E218860108860289828A83E0A3F5F0E0C5F012012B89828A83F0A3C5F0F0C5F0F5
:20346E0018E60886F0C0E0C0F012062F158115817F071201D1F07F071201D1E075F0007B7B
:20348E00107C0012017F60327F041201D1E075F0007B207C001200BE2400C5F03400C5F019
:2034AE00797E7AA412007C89828A83E0A3F5F0E0C5F05402C5F05400C5F045F070477F07C0
:2034CE001201D1E075F0007B087C0012017F60357F041201D1E075F0007B207C001200BEFC
:2034EE002400C5F03400C5F0797E7AA412007C89828A83E0A3F5F0E0C5F05402C5F05400E5
:20350E00C5F012014C45F070030235907F001201D1E0A3F5F0E0C5F054FFC5F054DFC5F0CA
:20352E007F001201D1F0A3C5F0F0C5F07F071201D1E07F061201D1F090AC97E054207003F0
:20354E0002358D74C075F0A2C0E0C0F0746675F05AC0E0C0F07F071201D1E075F000C0E0D6
:20356E00C0F0740375F000124FC17FFA12005474C075F0A2C0E0C0F0120CFE1581158102DB
:20358E0035DFE475F0807F001201D1F0A3C5F0F0C5F074C075F0A2C0E0C0F0747675F05ABC
:2035AE00C0E0C0F07F071201D1E075F000C0E0C0F0740375F000124FC17FFA12005474C09D
:2035CE0075F0A2C0E0C0F0121285158115810235FD0235FD90AC97E0542070030235FD7407
:2035EE008B75F05AC0E0C0F0120CFE158115817F041201D1E075F0007B087C0012010BC052
:20360E00E0C0F07F051201D1E075F0007B047C0012010BD004D0034BC5F04CC5F07F061207
:20362E0001D112006A4B7F001201D112006E4BC5F04CC5F07F001201D1F0A3C5F0F0C5F0AF
:20364E007F001201D1E0A3F5F0E0C5F07F080201EB7FF57EFF1201ED740175F0007F00122B
:20366E0001D1F0A3C5F0F0C5F078FB1200488601088602C001C002181818E60886F0C0E0CA
:20368E00C0F012305D158115817F021201D1F0A3C5F0F0C5F0D083D082F0A3C5F0F0C5F0BD
:2036AE007F021201D1E0A3F5F0E0C5F05400C5F05480C5F045F060030239E57F021201D1EB
:2036CE00E0A3F5F0E0C5F05400C5F0540FC5F07B087C001201197F041201D1F07F021201A8
:2036EE00D1E0A3F5F0E0C5F054F0C5F05400C5F07B047C001201197F051201D1F07F0212DA
:20370E0001D1E0A3F5F0E0C5F0540FC5F05400C5F07F061201D1F078F91200488601088672
:20372E000289828A8312007589828A83E012008C7B3D1200831201767027188601088602A8
:20374E0089828A83E0A3F5F0E0C5F02401C5F03400C5F0F9AAF089828A83E012008C120147
:20376E004C45F07003023789748E75F05AC0E0C0F0121285158115810239E578F9120048B4
:20378E00860108860289828A83E0A3F5F0E0C5F012012B89828A83F0A3C5F0F0C5F07F022B
:2037AE001201D1E0A3F5F0E0C5F05400C5F05440C5F045F0700302382D7F041201D1E075FD
:2037CE00F00090381E02009578F9120048E60886F0C0E0C0F07F021201D1E0A3F5F0E0C082
:2037EE00F0C0E01240A015811581158115817F001201D1F0A3C5F0F0C5F002382A74AC7598
:20380E00F05AC0E0C0F01212851581158102382AD6370600D637020000000B380239E590B2
:20382E00A47DE075F00090388D02009578F9120048E60886F0C0E0C0F0740475F000C0E02C
:20384E00C0F012051215811581158115817F071201D1F0A3C5F0F0C5F002389978F912007C
:20386E0048E60886F0C0E0C0F012062F158115817F071201D1F0A3C5F0F0C5F00238996A37
:20388E00380A003A38100000003A387F021201D1E0A3F5F0E0C5F05400C5F05420C5F0450B
:2038AE00F070030238E77F041201D1E075F000C0E0C0F07F051201D1E075F000C0E0C0F07D
:2038CE007F071201D1E0A3F5F0E0C0F0C0E0121EB97FFA1200540239D67F071201D1E0A312
:2038EE00F5F0E0C5F07B017C0012018D700302391274C175F05AC0E0C0F012128515811550
:20390E00810239E57F041201D1E075F000C0E0C0F07F051201D1E075F000C0E0C0F01220CD
:20392E000515811581158115817F091201D1F0A3C5F0F0C5F0740175F0007F061201D1126E
:20394E00006A7C0012010BF475F0007F091201D112006E5BC5F05CC5F07F091201D1F0A3F0
:20396E00C5F0F0C5F07F071201D1E0A3F5F0E0C5F07F061201D112006A7C0012010B7F0971
:20398E001201D112006E4BC5F04CC5F07F091201D1F0A3C5F0F0C5F07F041201D1E075F0AF
:2039AE0000C0E0C0F07F051201D1E075F000C0E0C0F07F091201D1E0A3F5F0E0C0F0C0E0A8
:2039CE00121EB97FFA120054E4F5F07F001201D1F0A3C5F0F0C5F07F001201D1E0A3F5F02D
:2039EE00E0C5F07F0B0201EB7FF77EFF1201ED78F91200488601088602C001C0021818180C
:203A0E00E60886F0C0E0C0F012305D158115817F021201D1F0A3C5F0F0C5F0D083D082F032
:203A2E00A3C5F0F0C5F0740175F0007F001201D1F0A3C5F0F0C5F0E4F5F07F071201D1F02E
:203A4E00A3C5F0F0C5F07F021201D1E0A3F5F0E0C5F05400C5F05480C5F045F06003023D90
:203A6E00717F021201D1E0A3F5F0E0C5F05400C5F0540FC5F07B087C001201197F04120183
:203A8E00D1F07F021201D1E0A3F5F0E0C5F054F0C5F05400C5F07B047C001201197F051236
:203AAE0001D1F07F021201D1E0A3F5F0E0C5F0540FC5F05400C5F07F061201D1F07F0412C5
:203ACE0001D1E075F0007B207C001200BE2400C5F03400C5F0797E7AA412007C89828A835D
:203AEE00E0A3F5F0E0C5F05401C5F05400C5F045F06003023B5A74C075F0A2C0E0C0F0747A
:203B0E00DF75F05AC0E0C0F07F041201D1E075F000C333C5F033C5F079F77A5312007C8916
:203B2E00828A83E0A3F5F0E0C0F0C0E0740375F000124FC17FFA12005474C075F0A2C0E098
:203B4E00C0F012128515811581023D7178F7120048860108860289828A8312007589828A0E
:203B6E0083E012008C7B3D12008312016E7003023B9374FC75F05AC0E0C0F0121285158167
:203B8E001581023D717F021201D1E0A3F5F0E0C5F05400C5F05440C5F045F07003023BF444
:203BAE007F041201D1E075F000903BE8020095E4F5F07F001201D1F0A3C5F0F0C5F0E4F50F
:203BCE00F07F071201D1F0A3C5F0F0C5F0023D71E47F051201D1F0023BF4BD3B0600BD3B7D
:203BEE0002000000DE3B7F021201D1E0A3F5F0E0C5F05400C5F05420C5F045F07003023C22
:203C0E00EC7F041201D1E075F000903CDD0200957F041201D1E075F000C0E0C0F07F05122C
:203C2E0001D1E075F000C0E0C0F07F041201D1E075F0007B207C001200BEC0E0C0F07F05A8
:203C4E001201D1E075F000C333C5F033C5F0D004D0032BC5F03CC5F0797E7AA412007C89F6
:203C6E00828A83E0A3F5F0E0C5F05401C5F05400C5F045F06005E4F5F08005740175F000D5
:203C8E00C0E0C0F0122DC37FFA1200547F071201D1F0A3C5F0F0C5F0023CE97F041201D100
:203CAE00E075F000C0E0C0F07F051201D1E075F000C0E0C0F01220051581158115811581D5
:203CCE007F071201D1F0A3C5F0F0C5F0023CE91E3C04001E3C00000000A93C023D627F0497
:203CEE001201D1E075F000C0E0C0F07F051201D1E075F000C0E0C0F01220051581158115C8
:203D0E008115817F071201D1F0A3C5F0F0C5F07F071201D1E0A3F5F0E0C5F07F061201D157
:203D2E0012006A7C001201197F071201D1F0A3C5F0F0C5F07F071201D1E0A3F5F0E0C5F093
:203D4E005401C5F05400C5F07F071201D1F0A3C5F0F0C5F0E4F5F07F001201D1F0A3C5F077
:203D6E00F0C5F078FB12004886010886027F071201D1E0A3F5F0E0C5F089828A83F0A3C5D5
:203D8E00F0F0C5F07F001201D1E0A3F5F0E0C5F07F090201EB7FF97EFF1201ED740175F0DB
:203DAE00007F001201D1F0A3C5F0F0C5F078F9120048E60886F05400C5F05480C5F045F0AF
:203DCE007003023DF374C075F0A2C0E0C0F0741275F05BC0E0C0F012515615811581158194
:203DEE00158102405978F9120048E60886F05400C5F0540FC5F07B087C001201197F021276
:203E0E0001D1F018E60886F054F0C5F05400C5F07B047C001201197F031201D1F018E608D1
:203E2E0086F0540FC5F05400C5F07F041201D1F074C075F0A2C0E0C0F07F021201D1E07541
:203E4E00F000C333C5F033C5F079F77A5312007C89828A83E0A3F5F0E0C0F0C0E01251569D
:203E6E00158115811581158178F9120048E60886F05400C5F05440C5F045F06003023F364C
:203E8E0074C075F0A2C0E0C0F074C075F0A2C0E0C0F012518415811581D004D0032BC5F064
:203EAE003CC0F0C0E0742275F05BC0E0C0F07F031201D1E075F000C0E0C0F0740375F000EB
:203ECE00124FC17FFA12005478F9120048E60886F05400C5F05420C5F045F06003023F3663
:203EEE0074C075F0A2C0E0C0F074C075F0A2C0E0C0F012518415811581D004D0032BC5F004
:203F0E003CC0F0C0E0742675F05BC0E0C0F07F041201D1E075F000C0E0C0F0740375F00085
:203F2E00124FC17FFA12005474C075F0A2C0E0C0F0742A75F05BC0E0C0F0125146158115E5
:203F4E00811581158178F9120048E60886F05400C5F05420C5F045F06003023F7F742C75D8
:203F6E00F05B7F051201D1F0A3C5F0F0C5F0023FFD90A47DE075F000903FF10200957F0287
:203F8E001201D1E075F0007B207C001200BE2400C5F03400C5F0797E7AA412007C89828A09
:203FAE0083E0A3F5F0E0C5F05402C5F05400C5F045F06007742F75F05B8005743475F05B73
:203FCE007F051201D1F0A3C5F0F0C5F0023FFD743975F05B7F051201D1F0A3C5F0F0C5F07E
:203FEE00023FFDDD3F0A008C3F100000008C3F74C075F0A2C0E0C0F074C075F0A2C0E0C083
:20400E00F012518415811581D004D0032BC5F03CC0F0C0E07F051201D1E0A3F5F0E0C0F01C
:20402E00C0E078F7120048E60886F0C0E0C0F0740375F000124FC17FFA120054E4F5F07F30
:20404E00001201D1F0A3C5F0F0C5F07F001201D1E0A3F5F0E0C5F045F0700302407F74C084
:20406E0075F0A2C0E0C0F01212851581158102408F74C075F0A2C0E0C0F0120CFE158115E3
:20408E00817F001201D1E0A3F5F0E0C5F07F070201EB7FF97EFF1201ED740175F0007F006F
:2040AE001201D1F0A3C5F0F0C5F0742775F0547F021201D1F0A3C5F0F0C5F078F9120048B0
:2040CE00860108860289828A8312007589828A83E012008C45F0602C18860108860289828B
:2040EE008A8312007589828A83E012008C7B2C120083120176600D7F021201D112007589E1
:20410E00828A83E0700302464C78F9120048860108860289828A8312007589828A83E01290
:20412E00008C7B2012008312016E700302415F18860108860289828A83E0A3F5F0E0C5F0DB
:20414E0012012B89828A83F0A3C5F0F0C5F00240C97F021201D112007589828A83E075F0BA
:20416E00007B207C0012016E70030241997F021201D1E0A3F5F0E0C5F012012B7F02120116
:20418E00D1F0A3C5F0F0C5F00240C97F021201D112007589828A83E075F0007B807C001276
:2041AE00017F70030242727F021201D1120075C001C00278F7120048860108860289828A64
:2041CE0083120075D083D082E075F00089828A8312006A120083120176700302423174C00F
:2041EE0075F0A2C0E0C0F0743C75F05BC0E0C0F018860108860289828A83E0A3F5F0E0C04B
:20420E00F0C0E0740375F000124FC17FFA12005474C075F0A2C0E0C0F012128515811581C3
:20422E0002464C7F021201D1E0A3F5F0E0C5F012012B7F021201D1F0A3C5F0F0C5F078F979
:20424E00120048860108860289828A83E0A3F5F0E0C5F012012B89828A83F0A3C5F0F0C577
:20426E00F00246497F021201D112007589828A83E075F00090462202009578F91200488686
:20428E000108860289828A8312007589828A83E012008CC0E0C0F01250701581158145F0C7
:2042AE00602478F9120048860108860289828A8312007589828A83E012008CC0E0C0F012F3
:2042CE0050A41581158145F0700302430178F9120048860108860289828A83E0A3F5F0E080
:2042EE00C5F012012B89828A83F0A3C5F0F0C5F002428802462E744775F0AC7F041201D143
:20430E00F0A3C5F0F0C5F0744775F0ACC0E0C0F0E4C0E0C0E0745075F000C0E0C0F0125087
:20432E00EA7FFA12005478F9120048860108860289828A8312007589828A83E012008CC0CF
:20434E00E0C0F01250701581158145F0602478F9120048860108860289828A8312007589FE
:20436E00828A83E012008CC0E0C0F01250891581158145F070030243FD7F041201D1120058
:20438E0075C001C00278F7120048860108860289828A8312007589828A83E012008CC0E062
:2043AE00C0F01250B815811581D083D082F07F041201D1E0A3F5F0E0C5F012012B7F04122D
:2043CE0001D1F0A3C5F0F0C5F078F9120048860108860289828A83E0A3F5F0E0C5F0120106
:2043EE002B89828A83F0A3C5F0F0C5F0024334E47F061201D1F07F061201D1E075F0007BA0
:20440E00077C0012017F70120244A77F061201D1E0047F061201D1F080DC744775F0ACC07C
:20442E00E0C0F07F061201D1E075F000C333C5F033C5F079677A5412007C89828A83E0A3C6
:20444E00F5F0E0C0F0C0E0125212158115811581158145F060030244A478FB120048E6082E
:20446E0086F05400C5F0540FC5F07B087C00120119C0E0C0F0740C75F000C0E0C0F07F0662
:20448E001201D1E075F000C0E0C0F0121EB97FFA1200540244A70244197F061201D1E075C3
:2044AE00F0007B087C0012016E70030244F774C075F0A2C0E0C0F0746F75F05BC0E0C0F050
:2044CE00744775F0ACC0E0C0F0740375F000124FC17FFA12005474C075F0A2C0E0C0F01238
:2044EE0012851581158102464C02462E78F9120048860108860289828A8312007589828ACB
:20450E0083E012008CC0E0C0F01250701581158145F0602478F91200488601088602898298
:20452E008A8312007589828A83E012008CC0E0C0F01250A41581158145F070030245D67884
:20454E00F9120048860108860289828A8312007589828A83E0C394307F061201D1F008E67E
:20456E000886F05400C5F0540FC5F07B087C00120119C0E0C0F07F021201D112007589821C
:20458E008A83E0C3948075F000C0E0C0F07F061201D1E075F000C0E0C0F0121EB97FFA1222
:2045AE00005478F9120048860108860289828A83E0A3F5F0E0C5F012012B89828A83F0A3B9
:2045CE00C5F0F0C5F002461F74C075F0A2C0E0C0F074A075F05BC0E0C0F078F51200488610
:2045EE000108860289828A83E0A3F5F0E0C0F0C0E0740375F000124FC17FFA12005474C05B
:20460E0075F0A2C0E0C0F01212851581158102464C02462E04439100884290000000FA44E6
:20462E007F021201D1E0A3F5F0E0C5F012012B7F021201D1F0A3C5F0F0C5F00240C97F00F0
:20464E001201D1E0A3F5F0E0C5F07F070201EB7FF97EFF1201ED740175F0007F001201D1C5
:20466E00F0A3C5F0F0C5F078F9120048E60886F07B207C001200BE2400C5F03400C5F079EE
:20468E007E7AA412007C89828A83E0A3F5F0E0C5F05401C5F05400C5F045F060030246BB1F
:2046AE0079477AACE489828A83F00249B778F9120048E60886F0C0E0C0F0740D75F000C0F3
:2046CE00E0C0F07405C0E0C0F0121EB97FFA12005478F9120048E60886F0C0E0C0F0740DAB
:2046EE0075F000C0E0C0F012200515811581158115815402C5F05400C5F07F051201D1F0FC
:20470E007F051201D1E0700302474574017F061201D1F078F9120048E60886F0C0E0C0F0F5
:20472E00740D75F000C0E0C0F07404C0E0C0F0121EB97FFA1200547F051201D1E0600302F8
:20474E0046BB744775F0ACC0E0C0F0744775F0ACC0E0C0F012518415811581D004D0032B2D
:20476E00C5F03CC5F07F021201D1F0A3C5F0F0C5F078FB120048860108860289828A83E057
:20478E00700302498418860108860289828A83E075F0007B807C0012019570030249351813
:2047AE00860108860289828A83E075F0009049260200957F021201D1E0A3F5F0E0C0F0C0C4
:2047CE00E074D475F05BC0E0C0F0E51875F0007B0A7C001200BEC0E0C0F0740375F0001222
:2047EE004FC17FFA1200547F021201D1E0A3F5F0E0C5F02402C5F03400C5F07F021201D131
:20480E00F0A3C5F0F0C5F002493278F9120048E60886F0C0E0C0F0740C75F000C0E0C0F06C
:20482E001220051581158115811581540FC5F05400C5F07F041201D1F07F021201D1E0A37B
:20484E00F5F0E0C0F0C0E07F041201D1E075F000C333C5F033C5F079677A5412007C8982AF
:20486E008A83E0A3F5F0E0C0F0C0E012515615811581158115817F041201D1E075F000C305
:20488E0033C5F033C5F079677A5412007C89828A83E0A3F5F0E0C0F0C0E0125184158115BC
:2048AE0081C39401C5F09400C5F07F021201D112006E2BC5F03CC5F07F021201D1F0A3C5A0
:2048CE00F0F0C5F00249327F021201D1120075C001C00278F7120048E60886F0C0E0C0F0CC
:2048EE0008860108860289828A83E0C3948075F000C0E0C0F0122005158115811581158178
:20490E00540FC5F05400C5F02430C5F03400C5F0D083D082F002493218489100C1479000DB
:20492E000000D5480249557F021201D1120075C001C00278F9120048860108860289828AC6
:20494E0083E0D083D082F07F021201D1E0A3F5F0E0C5F012012B7F021201D1F0A3C5F0F014
:20496E00C5F078FB120048E60886F012012B18F608A6F002477F78F9120048E60886F0C0A2
:20498E00E0C0F0740D75F000C0E0C0F07404C0E0C0F0121EB97FFA120054E4F5F07F001259
:2049AE0001D1F0A3C5F0F0C5F07F070201EB7FFC7EFF1201ED740175F0007F001201D1F091
:2049CE00A3C5F0F0C5F078F9120048E60886F05400C5F05480C5F045F07003024A0C744750
:2049EE0075F0ACC0E0C0F074D975F05BC0E0C0F01251561581158115811581024B4978F9D3
:204A0E00120048E60886F05400C5F0540FC5F07B087C001201197F021201D1F018E608869D
:204A2E00F054F0C5F05400C5F07B047C001201197F031201D1F07F021201D1E075F0007BD4
:204A4E00207C001200BE2400C5F03400C5F0797E7AA412007C89828A83E0A3F5F0E0C5F062
:204A6E005401C5F05400C5F045F06003024AC3744775F0ACC0E0C0F0740075F05CC0E0C0BD
:204A8E00F07F021201D1E075F000C333C5F033C5F079F77A5312007C89828A83E0A3F5F090
:204AAE00E0C0F0C0E0740375F000124FC17FFA120054024B49744775F0ACC0E0C0F07F02A8
:204ACE001201D1E075F000C333C5F033C5F079F77A5312007C89828A83E0A3F5F0E0C0F031
:204AEE00C0E01251561581158115811581744775F0ACC0E0C0F0741D75F05CC0E0C0F01227
:204B0E00514615811581158115817F021201D1E075F000C0E0C0F078F9120048E60886F06F
:204B2E00C0E0C0F012465D15811581158115817F001201D1F0A3C5F0F0C5F07F001201D157
:204B4E00E0A3F5F0E0C5F045F07003024B6F744775F0ACC0E0C0F012128515811581024BA8
:204B6E007F744775F0ACC0E0C0F0120CFE158115817F040201EB7FFA7EFF1201ED74C07534
:204B8E00F0A2C0E0C0F0741F75F05CC0E0C0F078F7120048E60886F0C0E0C0F0740375F028
:204BAE0000124FC17FFA12005474C075F0A2C0E0C0F0120CFE1581158178FB120048E60858
:204BCE0086F045F06007740475F0008003E4F5F07F001201D1F0A3C5F0F0C5F0E4F5F07FF4
:204BEE00021201D1F0A3C5F0F0C5F07F021201D1E0A3F5F0E0C5F07B087C0012017F702051
:204C0E00024C8D7F021201D1E0A3F5F0E0C5F012012B7F021201D1F0A3C5F0F0C5F080CB6E
:204C2E0074C075F0A2C0E0C0F0742575F05CC0E0C0F07F001201D1E0A3F5F0E0C0F0C0E036
:204C4E007F021201D1E0A3F5F0E0C0F0C0E0E4C0E0C0E0122DC37FFA120054C0E0C0F07480
:204C6E000375F000124FC17FFA12005474C075F0A2C0E0C0F0120CFE15811581024C117813
:204C8E00FB120048E60886F045F06007740575F0008005740175F0007F001201D1F0A3C5B9
:204CAE00F0F0C5F0E4F5F07F021201D1F0A3C5F0F0C5F07F021201D1E0A3F5F0E0C5F07B59
:204CCE00047C0012017F7020024D537F021201D1E0A3F5F0E0C5F012012B7F021201D1F08D
:204CEE00A3C5F0F0C5F080CB74C075F0A2C0E0C0F0742B75F05CC0E0C0F07F001201D1E0E0
:204D0E00A3F5F0E0C0F0C0E07F021201D1E0A3F5F0E0C0F0C0E012200515811581158115C2
:204D2E0081C0E0C0F0740375F000124FC17FFA12005474C075F0A2C0E0C0F0120CFE15817A
:204D4E001581024CD978FB120048E60886F045F06007740775F0008005740375F0007F00FB
:204D6E001201D1F0A3C5F0F0C5F0E4F5F07F021201D1F0A3C5F0F0C5F07F021201D1E0A351
:204D8E00F5F0E0C5F07B047C0012017F7020024E197F021201D1E0A3F5F0E0C5F012012B65
:204DAE007F021201D1F0A3C5F0F0C5F080CB74C075F0A2C0E0C0F0743175F05CC0E0C0F007
:204DCE007F001201D1E0A3F5F0E0C0F0C0E07F021201D1E0A3F5F0E0C0F0C0E01220051581
:204DEE0081158115811581C0E0C0F0740375F000124FC17FFA12005474C075F0A2C0E0C09A
:204E0E00F0120CFE15811581024D9F744775F0547F041201D1F0A3C5F0F0C5F078FB120011
:204E2E0048E60886F045F06007740675F0008005740275F0007F001201D1F0A3C5F0F0C57D
:204E4E00F079477AACE489828A83F07F001201D1E0A3F5F0E0C5F07B207C001200BE240017
:204E6E00C5F03400C5F0797E7AA412007C89828A83E0A3F5F0E0C5F05401C5F05400C5F0BB
:204E8E0045F07003024EBF7F001201D1E0A3F5F0E0C0F0C0E07F041201D1E0A3F5F0E0C0E3
:204EAE00F0C0E012465D1581158115811581024EDC744775F0ACC0E0C0F0743775F05CC0D3
:204ECE00E0C0F01251561581158115811581744775F0ACC0E0C0F0120CFE158115817F063A
:204EEE000201EB7FFE7EFF1201ED1201F8121DEF120205D2AF12089390A38BE06003024FFA
:204F0E003F744875F05CC0E0C0F0120CFE15811581747C75F05CC0E0C0F0120CFE15811567
:204F2E0081748175F05CC0E0C0F0120CFE158115811221951212BF740175F00045F0700367
:204F4E00024F9BE4A21792E0F51F7003024F65B297B297B297C217120FD17F001201D1F012
:204F6E00A3C5F0F0C5F07B007C001201767003024F987F001201D1E0A3F5F0E0C0F0C0E04F
:204F8E00121826158115811212BF024F4574A975F05CC0E0C0F0120CFE158115817F020215
:204FAE0001EB23F42581F81201B91252891201B902045E23F42581F886820886830802522F
:204FCE0089000000000000000000202020202000000000000000000000000000000000009A
:204FEE0000600101010101010101010101010101011818181818181818181801010101013F
:20500E0001010A0A0A0A0A0A02020202020202020202020202020202020202020101010118
:20502E0001010C0C0C0C0C0C040404040404040404040404040404040404040401010101C4
:20504E0000C2D578FB120048E6904FCFC2E79355F060027401A2D575F00092F065F075F0DA
:20506E00002278FB120048E6A2E7B3E4F5F092E02275F00280CB75F00480C675F00680C1A7
:20508E0075F01680BC75F01780B775F05780B2D2D575F05780AD75F01080A675F00880A1F1
:2050AE0075F001809C75F020809778FB120048E6C0E008E6C0E012508413D0F0D0E0500228
:2050CE0024E02278FB120048E6C0E008E6C0E012507F13D0F0D0E050E924202278F7120037
:2050EE0048868208868308860708088603088604EB4C600AEFF0A31BBBFFF51C80F222786C
:20510E00FB1200488682088683E4FBFCFFE0A3B42D030FE0A3C39430B40A005012FA740A21
:20512E0075F0001200BE2AFBE5F03400FC80E4EB8CF0DF030201432278F912004886820812
:20514E008683E0600DA380FA78F91200488682088683088601088602C9C582C9CAC583CA16
:20516E00E0A3C9C582C9CAC583CAF06003A380E8E5828583F02278FB120048868208868324
:20518E00E4F5F0FAE06009A30ABA00F805F080F4EA2278FB120048E60886F030F73A02018C
:2051AE004378F91200488603088604088605088606ED8EF012019B401CED8EF02278F9120C
:2051CE0000488603088604088605088606ED8EF012019B40E4EB8CF02278FB12004886031B
:2051EE0008860485FEF0E5017F0012017F600575F001E422EF0FF5F0A412017F70F6EF1452
:20520E0075F0002278F91200488682088683088601088602C9C582C9CAC583CAE0F5F0A3D9
:20522E00C9C582C9CAC583CAE0B5F0056009A380E37401500274FF02008C78FB1200488697
:20524E0082088683E075F0002278FB1200488682088683E0F5F0A3E0C5F02278F912004876
:20526E00868208868308E6F02278F9120048868208868308E608F0A3E6F0221253D0868265
:20528E0008868308E4FEFFE070061253D0E4F022B42551A3E0B42D05430780A3E0B43003BE
:2052AE0043074024D0B40A00500BCE75F00AA42EFEA3E080EEE0B46413E60886F030F708AD
:2052CE00430720120143A6F018F68003B4750543070A8021B478054307108019B46F10431C
:2052EE00070880111253D0F0A31253D0A38095B462624307027A00C004C005C006C007AB4C
:20530E000753031F7C00E60886F01200D8A6F018F6EDD007D006D005D0042430B43A0040D0
:20532E00022407C0E00AE645F070CC1253D0A902EF30E505742DF0A30A1253D9D0E0F0A389
:20534E00D9FA0808EF30E7A1EAC39E509C7420F0A30A80F4B4630DAA011253D01253D9E6B1
:20536E00F0A380DEB47331C082C08386820886837A00E06004A30A80F986831886821253C6
:20538E00D01253D91253D0E0A31253D06004F0A380F2D005D00480AAB4691B86017A00E7A8
:2053AE006004090A80F91253D01253D98601E76091F009A380F8F97A011253D01253D9E939
:2053CE00809ECDC583CDCCC582CC22EE601A8FF020F715C002EAC39E500C742030F6027412
:2053EE0030F0A30A80EFD002228054845488548D549154955499549E5410E020E030E00059
:20540E00E050E060E070E040E0080008000F000400080008000F00040089882F87862F8B71
:20542E008A20912085843A83823A81802E900000000000000000000000898887868B8A206F
:20544E0085848382818090000000000000000000000000000000000000A254A654AA54AE03
:20546E0054B254B654BA5400004144494F3020003F5541493000414F3000434C4B300044E3
:20548E0050300041493100414F3100434C4B31004450310053554E004D4F4E005455450064
:2054AE0057454400544855004652490053415400436F6E736F6C6520737461747573206627
:2054CE006C61677320253032780A00205472616E733A20204865616420253032782C20541B
:2054EE0061696C20253032782C2043747220253032782C204D617820253032780A002052A8
:20550E0065633A202020204865616420253032782C205461696C20253032782C2043747200
:20552E0020253032782C204D617820253032780A0030313233343536373839414243444547
:20554E0046003030200020002A2A2A2042616420636865636B73756D3A202532780A002AE2
:20556E00000A002A2120004F4B0A003E002A2A2A204E6F2061646472657373207374726983
:20558E006E672E2E2E0A004E657420616464726573732069732025730A004E65742061649D
:2055AE006472657373205B25735D002E2020537461636B207573656420253032782F253074
:2055CE0032782E0A004572726F7220666C61677320253032782E20204E6574776F726B200D
:2055EE00636865636B73756D206572726F72732025750A004C6F6767696E67206D6F64653D
:20560E002069732025750A004E6574206D6F64652069732025750A002A2A2A204E20636D34
:20562E00642073796E746178206572726F720A002A2A2A20556E6B6E6F776E20636F6D6D83
:20564E00616E643A205B25735D0A0054305469636B732025750A002A2A2A20496E76616C77
:20566E00696420514120636F6D6D616E640045534554002A2A2A20556E6B6E6F776E20635C
:20568E006F6D6D616E640A00417661696C61626C6520636F6D6D616E6473202876616C7583
:2056AE00657320696E20646563696D616C20756E6C657373206E6F746564290A0020413D59
:2056CE00737472696E672020202B20736574206E6574776F726B206164647265737320746A
:2056EE006F20737472696E670A002044202020202020202020202A20646973706C61792068
:20570E00696E7465726E616C20737461747573207661726961626C65732028736F6D652065
:20572E00696E20686578290A002045202020202020202020202A2073686F7720616E6420C9
:20574E00636C656172206572726F7220666C6167730A00204C206E20202020202020202099
:20576E0020736574207265706F7274696E67206D6F646520286269746D6170706564290ABF
:20578E0000204E206E202020202020202A2B20736574206E6574776F726B206D6F64650A65
:2057AE00002051202020202020202020202020717565727920696E707574730A0020524530
:2057CE005345542020202020202020706572666F726D20706F7765722D6F6E2072657365AE
:2057EE007420696E697469616C697A6174696F6E0A00205320202020202020202020202022
:20580E00736574206F75747075742076616C7565730A002B206D61726B73206E6574776FED
:20582E00726B2D6F6E6C7920636F6D6D616E64730A002A206D61726B73206465627567671C
:20584E00696E6720636F6D6D616E64730A005772697465202530327820746F206164647298
:20586E0065737320253034780A005265616420253032782066726F6D20616464726573732F
:20588E0020253034782025730A0066616B65640000496E697469616C697A696E6720646548
:2058AE007669636520696E666F726D6174696F6E0A00202E2E2E25733A2000617373756D9E
:2058CE0065206E6F7420696E7374616C6C6564000A007479706520697320005344413038DC
:2058EE0031300041444330383038006E6F7420696E7374616C6C6564002C20454F432074B9
:20590E00657374733D257500617373756D65204144433038303800617373756D6520696E18
:20592E007374616C6C65642C20736574206F75747075747320746F203030006E6F74206937
:20594E006E7374616C6C656400696E7374616C6C6564002C20696E7420656E61626C6564A0
:20596E00002C203234206872206D6F64652C2073746172746564002C20696E74206469736E
:20598E0061626C65642C206E6F742073657420757000617373756D6520696E7374616C6C4E
:2059AE0065642C206368616E6E656C7320302D31203D20696E7075742C2032203D206F753E
:2059CE0074707574002A2A2A20257320454F4320696E616374697665206265666F72652099
:2059EE00636F6E766572740A002025732E2575203D20253032780A002A2A2A2042616420C3
:205A0E00646576696365206E616D65205B25735D0A005B446576696365202573002C2063BB
:205A2E0068616E6E656C203D202575000A2A2A2A20426164206368616E6E656C20666F72BC
:205A4E002025733A2025750A002C20616C6C206368616E6E656C73002C2062697420494459
:205A6E00203D2025755D0A000A2A2A2A20426164206269742049443A2025750A005D0A007A
:205A8E002A2A2A2053657420636F6D6D616E64206D697373696E6720646174610A002A2AFD
:205AAE002A204D697373696E67206368616E6E656C0A002A2A2A204269742076616C7565B7
:205ACE00206D7573742062652030206F7220310A002A2A2A20446576696365202573206E08
:205AEE006F7420696E7374616C6C65640A002A2A2A2043616E6E6F74207365742076616CFB
:205B0E0075650A002A2A2A20426164206465766963650A002E2575002E2575003D002575ED
:205B2E0000253034780025303278002575002A2A2A2A20536570617261746F72206D6973DB
:205B4E006D61746368206174205B25735D2C20636C6F636B206D6179206265206261640ACE
:205B6E00002A2A2A2A20496E76616C696420646179206F66207765656B205B25735D2C20AD
:205B8E00636C6F636B206D6179206265206261640A002A2A2A2A20496E76616C6964207429
:205BAE00696D6520737472696E67206174205B25735D2C20636C6F636B206D6179206265DA
:205BCE00206261640A0025303375002A2A2A2043616E6E6F742073686F772074696D652C8C
:205BEE00206261642064657669636520636F64650A002A2A2A204465766963652025732035
:205C0E006E6F7420696E7374616C6C65640A003D00514125643D00253034782000253034FC
:205C2E0078200025303278200030303030303020303030303030303030000A4144494F2D5B
:205C4E004C696E6B204E6574776F726B656420416E616C6F672026204469676974616C201F
:205C6E00492F4F2C2056657273696F6E2000312E3164000A2020436F7079726967687420E6
:205C8E003139393220436972637569742043656C6C61722C20496E632E0A002D2D2D204630
:155CAE00656C6C206F75742074686520626F74746F6D210A00EB
:00000001FF
